:1000000042C084C15BC05AC059C058C057C056C016
:1000100055C054C053C052C051C050C04FC04EC054
:100020004DC04CC04BC04AC049C048C047C046C084
:1000300045C044C0090212000101008019090400F2
:1000400000000000000012010101FF000008C016BE
:10005000DC050101010200010E03550053004200BE
:100060006100730070001C037700770077002E009A
:10007000660069007300630068006C002E00640075
:1000800065000403090411241FBECFEFD2E0DEBFD8
:10009000CDBF11E0A0E0B1E0ECE7FDE002C00590CB
:1000A0000D92A230B107D9F711E0A2E0B1E001C092
:1000B0001D92A234B107E1F744D65FC6A1CF1F93CA
:1000C000CF93DF9360913C01662359F1635067FD44
:1000D0006CC0C2E0D1E0C0913601CF5F20E010E8F3
:1000E000809139018D3209F465C08091180187FD36
:1000F00009C0CE0187D52FEF821709F49FC0811167
:1001000020E010E010931801922F2093010110922B
:100110003C019F3F51F483B1837089F11092190122
:10012000E3C0909101019F3FB1F38091000184FFF2
:10013000F2CF692F9930B8F5961B909301011BE41B
:100140008091180180FD13EC8F5F80931801ACE261
:10015000B1E087FD60C0662309F058C060E070E040
:10016000C62F693008F446C02EE18FEF809301015D
:1001700010932B012093000183B1837079F6809155
:100180001901882309F0B0C094E683B1837009F0A7
:10019000ABC09150D1F781E08093190190933D015C
:1001A00090933801A1C068E0C7CF909101011092EF
:1001B0003C01AFCF683009F0A5CF8881807609F087
:1001C00056C044E351E0209334018981882309F02B
:1001D00041C02093350122E050933B0140933A0106
:1001E0008F81882309F08ECF8E81821708F08ACF05
:1001F000282F88CF8CE291E02CD22C2F2C5FC83096
:1002000008F0B6CF9FEF90930101B2CFCD01BDD4DE
:10021000682F7727A5CFE0913A01F0913B0186FF47
:1002200012C0962F03C084918D9331969150D8F7C8
:10023000F0933B01E0933A01772792CF8EE18093D0
:10024000000110E05FCF962F02C081918D939150F5
:10025000E0F7EECF8530B9F08630C9F0883039F15B
:10026000893049F18A3009F0BBCF21E0B5CFCE010A
:10027000A3D3282F8F3F09F0B3CF888187FF41CFC9
:100280002E8110E03FCF8A8180933D01A9CF10ECF1
:100290008B818130A1F08230B1F0833009F0A0CFA2
:1002A0008A818823A1F442E850E024E095CF4FE30F
:1002B00051E021E091CF8A8180933F0191CF46E4C4
:1002C00050E022E189CF44E350E022E185CF813044
:1002D00039F0823009F084CF48E550E02EE07CCF41
:1002E00046E650E02CE178CFDF91CF911F91089541
:1002F00082E091E0809337010B96809336018091E4
:100300006900836080936900E89A08950F930FB79E
:100310000F93189BFECF189B06C0189B04C0189B18
:1003200002C0000000C01F933F932F9331E012E002
:1003300003B1102710FD32E0102F3A95C9F700FDE8
:10034000E3C003B1102720E010FB20F9DF9313B1C5
:10035000012700FB21F9CF93C091370103B110278A
:1003600010FB22F93BE0D1E04F9313B1012700FBD2
:1003700023F94FEF000055C0189BFECF189B06C015
:10038000189B04C0189B02C0000000C0DF9100C091
:10039000CDCF13B1137079F14F7D206213C003B13B
:1003A000037049F14F7B206415C0037021F1102FB9
:1003B000206803B119C003B10370E9F04E7F2160DA
:1003C00018C039F303B10370B1F0102710FB26F900
:1003D000223028F313B1012700FB27F94227499364
:1003E0004FEF03B1243008F3102710FB20F9297FC9
:1003F00011F313B11370E1F1012700FB21F9237F01
:10040000F1F003B10370A1F1102710FB22F9277E50
:10041000E1F013B1012700FB23F93A9541F12F7C5C
:10042000D1F003B1037021F1102710FB24F92F79CB
:10043000C1F013B1012700FB25F92F73C2CF13B10F
:100440001370B1F04D7F2260DCCF03B1037081F0F7
:100450004B7F2460DECF13B1137051F0477F2860CB
:10046000E0CF03B1037021F04F7E2061E2CF3BC0AB
:100470003C2FC09137013C1B01E033300CBB98F19D
:1004800008811981412F1F77209138010D3279F1B0
:10049000013E69F10936C1F00777033421F5109167
:1004A0003E01112301F100913C010030C1F53430CF
:1004B000C2F130933C011093390100913601C09391
:1004C0003601009337012DC0121769F430910001F5
:1004D00034FD23C00AE500930001CBE2D1E025C042
:1004E000002700933E014F91CF91DF910DC012176D
:1004F000B9F700933E010AE5009300014F91CF91B7
:100500000CB300FD39CFDF9101E00CBB2F913F917F
:100510001F910F910FBF0F911895432F03C04AE50C
:1005200001C042EDC4E1D0E032E05F9353E0289A8D
:1005300005B1209A219A20E80FC0052710E005B9DF
:1005400010C0052710E0089405B913C0052710E076
:1005500015C0052710E019C020FF052705B927950C
:1005600017951C3F50F720FF0527279505B91795CC
:100570001C3F38F720FF05272795179505B91C3F25
:1005800028F720FF0527279517951C3F05B908F781
:1005900000C0499120FF052705B9279517951C3FF5
:1005A00080F520FF0527279505B917951C3F68F5AD
:1005B00020FF05272795179505B91C3F58F520FF03
:1005C0000527279517951C3F05B938F5242F3A952F
:1005D00019F60C7F5F9105B932E03A95F1F7109169
:1005E0003D01C651D04011F010933801016014B1A3
:1005F0001C7F05B90C7F4F91CF9114B905B9DF91DC
:1006000083CF052710E005B9CACF052710E008946D
:1006100005B9CDCF052710E0CFCF052710E0D3CF08
:10062000A82FB92F8FEF9FEF41E050EA615070F093
:100630002D9138E0722F782796958795269570FF33
:1006400002C0842795273A95A9F7F0CF8095909519
:100650000895E6DF8D939D9308953B98439A00009B
:100660000000339904C082E58CBD1DBC08953A9A00
:10067000429800000000339B07C082E58CBD81E0FA
:100680008DBD3A98429A089583E58CBD1DBC3A9879
:10069000429A0895882339F48FE793E090934101BB
:1006A0008093400108958CE993E0909341018093F9
:1006B0004001089596B586B5891B8C30E0F3089506
:1006C0002C9A3D9A459884B18C6284B92A982D98C9
:1006D000F1DF2A9AEFDF2A98809140019091410141
:1006E0008C59934009F00895B8DF089584B1837D53
:1006F00084B985B1837D85B93D981CBC08950F935D
:100700001F93CF93C82F00E017E00CC02B98CC0F9D
:10071000000F1C990F5FCEDF2D9ACCDF2D98115062
:1007200017FD04C0C7FFF2CF2B9AF1CF802F992776
:10073000CF911F910F9108958EBD0DB407FEFDCF8F
:100740008EB5992708951F93CF93CFE103C0C15071
:10075000CF3F51F1E0914001F09141018CEA0995C0
:10076000E0914001F091410183E50995E09140015C
:10077000F091410180E00995182FE0914001F0913E
:10078000410180E00995133591F01CBC2D9A92DF50
:100790002D9890DF80914001909141018C599340B8
:1007A000B1F65BDFC150B0F681E090E002C080E0BE
:1007B00090E0CF911F9108950F931F938C0181704A
:1007C000880F880F880FE0914001F091410180620D
:1007D0000995C801892F99278695E0914001F091EC
:1007E0004101099516950795E0914001F09141016D
:1007F000802F0995E0914001F091410180E0099539
:1008000099271F910F9108950F931F93CF93DF9313
:10081000EC01062F142F8170880F880F880FE0914C
:100820004001F091410180640995CE01892F9927FB
:100830008695E0914001F09141010995CE01969590
:100840008795E0914001F09141010995E0914001C7
:10085000F0914101802F09951123A9F00F3789F0FC
:100860001EE106B5CE01A8DF8F3769F486B5801B7F
:100870008D3310F006B511501123A1F781E090E0FF
:1008800004C08FE08CD080E090E0DF91CF911F9189
:100890000F9108950F931F93CF93DF93EC01162FC1
:1008A000E0914001F09141018CE40995CE01892F3E
:1008B00099278695E0914001F09141010995CE017B
:1008C00096958795E0914001F09141010995E0915D
:1008D0004001F091410180E009951F3F89F01EE140
:1008E00006B5CE0169DF8F3F69F486B5801B8D3375
:1008F00010F006B511501123A1F781E090E004C07B
:100900008FE04DD080E090E0DF91CF911F910F916B
:1009100008950F931F938C01E0914001F0914101E4
:1009200080EA0995812F9927E0914001F0914101DA
:100930000995E0914001F0914101802F0995E091E6
:100940004001F091410180E0099599271F910F9195
:100950000895FF920F931F938C01F62EE0914001B2
:10096000F091410180EC0995812F9927E091400198
:10097000F09141010995E0914001F0914101802FF2
:100980000995E0914001F09141018F2D09958EE18B
:1009900006D080E090E01F910F91FF900895382FCE
:1009A00020E0231740F496B586B5891B8C33E0F31D
:1009B0002F5F2317C0F308951F93CF93DF93EC01AC
:1009C00010E089818130A1F0823009F489C0833040
:1009D00009F489C0843091F0873009F467C085300C
:1009E00009F4C3C0863039F1883009F0C2C09DC017
:1009F000329B812F4FDE64DE4198BBC08B819927EB
:100A0000982F88272A813327822B932B90932601B6
:100A1000809325018F819927982F88272E8133274E
:100A2000822B932B90931B0180931A0182E0809379
:100A30001C011FEF9EC08B819927982F88272A8140
:100A40003327822B932B90932601809325018C8151
:100A5000482F552750932801409327012D812F704F
:100A6000209329018D819927807F9070829592959E
:100A7000907F9827807F9827840F951F9093280157
:100A80008093270120FF04C08091270180932A01D1
:100A90008F819927982F88272E813327822B932B9C
:100AA00090931B0180931A0181E0C1CF8B8199271C
:100AB000982F88272A813327822B932B9093260106
:100AC000809325018F819927982F88272E8133279E
:100AD000822B932B90931B0180931A0183E0A7CF65
:100AE00005DE419A46C0E0914001F09141018A81C2
:100AF000099580931D01E0914001F09141018B81A6
:100B0000099580931E01E0914001F09141018C8193
:100B1000099580931F01E0914001F09141018D8181
:100B200009958093200114E024C08B819927982F88
:100B300088272A813327822B932B90932601809339
:100B400025011092280110922701109329018F810D
:100B50009927982F88272E813327822B932B9093C8
:100B60001B0180931A0184E062CFEDDD80931D01AB
:100B700011E08DE191E090933B0180933A01812F48
:100B80009927DF91CF911F910895EF92FF921F93C4
:100B9000CF937C01162F90911C01892F82508230B7
:100BA00050F5C0E0C617C0F01FC08091250190919C
:100BB0002601AFDEF701EC0FF11D80838091250146
:100BC0009091260101969093260180932501CF5F95
:100BD000C11750F490911C01923039F78091250192
:100BE00090912601E9DDE6CF183010F410921C0137
:100BF000812F992702C08FEF90E0CF911F91FF9036
:100C0000EF900895BF92CF92DF92EF92FF920F93F1
:100C10001F93CF93DF936C01E62EBB2440911C0100
:100C2000413019F0443009F080C0FF24FE1408F070
:100C300079C0413009F049C0809127019091280185
:100C4000892B09F04EC0CF2DDD27FE01EC0DFD1DD7
:100C500060818091250190912601D6DD80911A0155
:100C600090911B01019790931B0180931A01892B8E
:100C7000D9F410921C018091290181FF13C0809149
:100C80002A01282F332780912701909128012817C6
:100C9000390741F0CC0DDD1D6881809125019091CF
:100CA0002601F8DDC1E0BC2E80912501909126013E
:100CB00001969093260180932501F394FE1490F5FC
:100CC00040911C01413009F4B7CFCF2DDD27FE0143
:100CD000EC0DFD1D6081809125019091260139DE8A
:100CE000BDCFCF2DDD278E010C0D1D1D40E0F8017D
:100CF0006081809125019091260186DD80912A01F5
:100D0000815080932A01882309F0A8CFF8016081DF
:100D10008091250190912601BDDD8091270180936E
:100D20002A019CCF8B2D992702C08FEF90E0DF9195
:100D3000CF911F910F91FF90EF90DF90CF90BF90D8
:100D40000895CFEFD2E0DEBFCDBF1BB815B88BEF53
:100D50008AB98FEF84B990E09150F1F78150D9F7BB
:100D600084B993E097B98EEF88B995BD81E092DCA4
:0C0D7000BFDA7894A4D9A3D9FDCFFFCF3F
:020D7C005AFF1C
:00000001FF
